:1000BE002227E22F0DD0293020F4332730832395C9
:1000CE00F8CF408323EB31E03A932A934AE0BBC743
:1000DE00FF27ED54FE4F08951127E12FF9DF008120
:1000EE00193020F4002349F41395F7CF102F163E44
:1000FE0011F0173E11F4012F089500270895FDDE2B
:10010E0003EB11E028D035D0063E31F403EB11E0BD
:10011E0024D02FD0073ED1F0AA27BB2780E092E053
:10012E002AD080F420D025D0002351F0063E19F4B9
:10013E00A39525D005C0B3958093E9019093EA016C
:10014E000A96EECFA13021F4B13011F401E001C0D6
:10015E000027E4E0E3CE18D01BC016D00091E901D1
:10016E001091EA01089503EB11E00ED0082F192F1C
:10017E0008954ED7B1CF873F0FE190070895809332
:10018E00E7019093E80108951A930A934AE00895BF
:10019E000091E7011091E8010895B1DE80E092E050
:1001AE00EADF88F4E0DFE5DF002359F000270A30AC
:1001BE0030F41FEFE02F8CDF10830395F8CFD3DFE1
:1001CE0042D70A96EDCF07D00AE00CD010D012D04D
:1001DE006FDFE2E0A5CE00E012E00093E70110939E
:1001EE00E80108950093E9011093EA01089546EE9F
:1001FE00CFDF5ECF47EEB2CF82DF002309F4CDDF33
:10020E0009EA11E0AADF1FD7E9EEF1E01AD020D0FB
:10021E00073F1F4118F000E012E0E4DF19D02091F3
:10022E00E7013091E8010217130749F4E7EEF1E018
:10023E0008D0AEDF073F1F4108F0CDDFD8DFDADF91
:10024E0037CF00811181065F1F4F00831183089500
:10025E0085CF55DE8091E7019091E8010A968BDFFC
:10026E0010F080E092E0F4DF8017910721F047DF75
:10027E00002319F492DF00270EC009EA11E075DFA2
:10028E00C7D609EA11E067DFDED646EE082F192F32
:0A029E000FDF75DF01E0E2E043CE60
:1002A800B09B0AC000919E010330A8F400919E0102
:1002B800039500939E01089500919E01033040F03C
:1002C800EDEBF1E0008111810F5F1F4F0083118377
:0802D800002700939E01089528
:1002E000002311F00A95FCCF089503D0949804E000
:1002F000F7CF949A04E0F4CF949893988B9A08954A
:10030000FBDF939AF6DF9398F5DF94980895F4DF76
:10031000F0DF939AF9CF8A938B988827839B8FEF8E
:10032000E4DF8B9A082F899108958A938B98882708
:10033000839B8FEFDADF082F8991089593988B9A2A
:10034000D4DF8B980895939A8B9ACFCFDFDD802FDF
:1003500098E09A9501E0492F60DD082311F0939A07
:1003600001C09398C2DF9923A1F7E2E0E0CDCEDD92
:1003700088E08A95839B05C001E0482F4EDD902BD5
:1003800005C001E0482F49DD00959023AEDF8823AA
:1003900081F7092FE2E0CBCDB9DDB2DF0AD0918140
:1003A000892F80688E7F08D004D0008106D0E2E0DB
:1003B000BECDE0E6FF270895082FC8DFACCFA4DD4F
:1003C0000091A40102FF21C0F4DF9181892F90FDEB
:1003D000E3DF8068816094DF082FB8DFA6DFC7DF26
:1003E00011270093BF011093C001E3DF1181812F1A
:1003F00080304CF4A3DFBBDFEFEBF1E020813181F3
:10040000302B208331839FDF82DFE4E08ECD7CDDE3
:10041000802F912F0091A40102FF0BC0BDDFC9DF27
:10042000B181AB2FB0FDC8DFA03014F4092FC5DFB8
:060430006EDFE4E07ACD6E
:10043600F8940EBB1FBBE09A0DB37894089562DD65
:10044600802F912FA42FE02FF12F319729F001E073
:1004560010E0EEDF063E49F48EBB9FBBADBBF894C1
:10046600E29AE19A7894E199FECFE3E05CCD46EE1C
:0E04760001E010E0E4CF442701E010E0E0CF09
:100484000091E40101FF1AC00091C9011091CA0151
:100494002091CB013091CC010217130759F40027A6
:1004A4000093C9010093CA010091DF010260009327
:1004B400DF010895E9ECF1E004D006D00895E5ECFD
:1004C400F1E00081118108950F5F1F4F00831183B4
:1004D40008950091E40100FF29C029D00027107C71
:1004E400003020E8120749F427D02F7333272BD08C
:1004F4000F7320173040D1F414C00030104441F47D
:100504001BD0377020D017702017310779F409C039
:100514000ED01F732091C5013091C6010217130735
:1005240029F40091DF0101600093DF010895009137
:10053400C7011091C80108952091C7013091C801E5
:100544000895008311830091C5011091C601089597
:100554000A921A922A923A920A931A932A933A93F3
:100564004A935A936A937A93EA93FA93FFB7FA9366
:10057400789406E010E05DDF0093A40107E010E04A
:1005840058DF00939C01AFD00091A40101FD8ADEE5
:1005940080D576DFEAE8F1E094DF228133810050F0
:1005A400104C2F4F3F4F54D0228333838ADF228154
:1005B4003381003412442F403040C8F182DF22815D
:1005C4003381005412442F40304042D0228333837D
:1005D40000918E01039500938E0100918E010C33DE
:1005E40030F1002700938E016ADF6EDFE091C501D0
:1005F400F091C601EF73FF27FC97C0F060DF007C29
:1006040027D05FDF005C1F4F9CDF1770165070F01F
:1006140058DF0F73187F1CD054DF185F92DF185314
:1006240028F000270093C5010093C60152DFF99119
:10063400FFBFF991E9917991699159914991399162
:100644002991199109913990299019900990189537
:10065400008311830895102F1F70007F202F26958B
:10066400269526950695200F022F010F0895102F29
:1006740000271A3018F01A50005FFBCF010F0895BD
:1006840013D400918F01E7DF00938F010091900153
:10069400E2DF0093900100919101DDDF009391016D
:1006A400009192010A950093920100919101112702
:1006B40046E0CBDB202F312F0091920111274BE034
:1006C400C4DB200F311F009190011127200F311F2F
:1006D400F89400918F0100938E012093C50130930B
:0606E400C60178940895A0
:02000C00A3C28D
:1006EA0000919C01093018F008E000939C01002752
:1006FA0000939D0111E020919C010217F9F02091CD
:10070A009D01212B20939D0139B33123209193011F
:10071A002123321769F01AD020812395208316D01D
:10072A002081233040F020919301212720939301C7
:10073A0022270CD02083110F0395DDCF00919D0154
:10074A00109193011023109393010895E02FFF272E
:06075A00EC56FE4F08956D
:10076000D1DB04E025D0A02F05E022D0B02F1896D1
:100770008827A13002E0B00790F404E0402E552411
:100780004A165B0640F4042D152D55DE800F0FEF41
:10079000401A500AF5CF03E00BD0081711F006EE0F
:1007A00001C000270093A301082FE6E0BCCB02E0C4
:1007B00010E041CE06EE0093A201F9DF063E19F0EB
:1007C00059DE46EE01D0089502E010E03BDE56CE41
:1007D00000270093A2010091A40103FD06C0E7DFFA
:1007E000002319F047DE4427EFDF08950091A301AD
:1007F000063E11F402E008950091A201063E11F4B4
:100800000027089501E008950091A601023031F417
:1008100009D012D010933B0102E009D000270093C9
:10082000A60108950091A00100933A010895009354
:100830007F010093800108950091A0011091A10112
:1008400008958A930DDD013069F400270A3040F4E1
:1008500035D0E755FE4F31D035D010830395F6CF14
:1008600003E014C00091A601002311F0CDDF13C0F6
:100870000CE08827003118F4E02F0FD0FBCFB6DF53
:100880000093420100270093430101E000937F01A0
:100890000AE0009380018991089518D01081E82F13
:1008A000E65CFE4F108311D020813181E82FE55C9A
:1008B000FE4F308303958E5F08951081E02FFF2750
:1008C000089508D0E65CFE4F0895E02FEE0FE05A41
:1008D000FF270895E0912201FF27EE0FFF1F0895E3
:1008E0008A930091A601002311F08EDF47C00027F4
:1008F0008827003118F4E02FD0DFFBCF002780E2FB
:100900008F32D8F4F894DADFEE0FFF1FE354FE4F76
:100910001081E82FFF27D6DF1083D0DFEE0FFF1FF7
:10092000E354FE4F20813181E82FFF27E55CFE4F25
:100930003083789403958E5FE3CF64D40091CD012A
:1009400000936A010091CD011091CE0110936B01CB
:100950000BB300936C0105B300936D010AB30093D0
:100960006E0104B300936F0141DF00937001002713
:100970000093710105D008E30093800189910895E7
:1009800001E000937F01089510932301A3DFE55C4C
:10099000FE4F008110912401089500912201003141
:1009A00038F438D0E091220191DF0083218308954B
:1009B00000912201083148F4F8942CD08BDFE356E3
:1009C000FE4F00832183789408950091220108311D
:1009D00031F420D00093CD012093CE0108950091F1
:1009E0002201093139F4009123010BBB009124014C
:1009F00005BB0895009122010A3139F400912301C9
:100A00000ABB0091240104BB0895BADF00270093BC
:100A100080010895209124010091230108958A9373
:100A20008091A60100270093A6015ADF8093A601BA
:100A300000912301003861F0009123010F3740F04D
:100A400040DF00811091230110239EDF102307C097
:100A500038DF008110912301102B96DF102B1093AB
:100A600024019BDF8991089520912301322F009169
:100A70002201202F002710912401011740F41EDFCE
:100A8000E20FF31F1ADF1EDF10830395F4CF78DF28
:100A90000091240100938001089514D022E0309148
:100AA0008501231708F0B1CFE22FFF27EE5DFE4F3F
:100AB0003081E22FFF27E00FF11F3297308323951B
:100AC000EECFA3CF00912301102F20912201022FFE
:100AD000089514D0AA2700912401A01740F416D03D
:100AE000AADCEA2FFF27EEDE0083A395F4CF48DFD0
:100AF0000091240100938001E3E018CA06DA809196
:100B00002301982F00912201802F08950A2F112789
:100B1000080F191F0895F2DFA2E000918501A017C8
:100B200058F4EA2FFF27EE5DFE4F4081EFDF0250C1
:100B3000104088DCA395F1CF23DF0027DBCFC2DF95
:100B40002AE331E03A932A934091240168D29FCF5F
:100B5000B9DF24E231E03A932A9340918501425073
:100B600079D253CF4091220101E010E06BDC4DCFF0
:100B7000F89400918E0100933A010091C501009311
:100B80003B010091C5011091C60110933C0178947E
:100B9000F7DE03E0009380010895F89400912201AC
:100BA00000938E0137DF11270093C5012093C60102
:100BB0007894E6DE10938001089578D100918F013A
:100BC00000933A010091900100933B010091910143
:100BD00000933C010091920100933D01D1DE04E0BD
:100BE00000938001089501D010CF0091220100935D
:100BF0008F01009123010093900100912401009343
:100C00009101009125010093920167C1D3DDA8DD18
:100C100009DE12DE10933B01B3DE02E00093800197
:100C20000895D6DD9DDDF1CE36D5F2CFDEDFF89426
:100C300009B70F7709BF43987894E6E8F1E0E53EFD
:100C400001E0F007002718F400833196F8CF003157
:100C500028F43BDEF083F1830395F9CFB8D0AADD09
:100C6000F89409B7006809BF439A7894D1CF2091CE
:100C700023010091220111270093E5012093E60151
:100C800098CF002711270093E5010093E60191CF4B
:100C90000091E50100933A010091E5011091E60110
:100CA000B9CFC0DDC9DDB6CF5BDD00933A0101E00D
:100CB000BEDD0895F89400917C0100304CF5009160
:100CC000820100FD25C000917C01007C00937C0125
:100CD0007894E0917B01FF27EE0FFF1FEC58FF4F48
:100CE000C895002D3196C895E02FF02D0995F89400
:100CF0000091820101600093820100917F011091B7
:100D00007C01102B10937C010091800100937E01E7
:040D10007894089536
:1000780021047004CD040F0534054D0569058B0571
:100088009F05A805B205B805CD05DD05F3050606EB
:100098001106140616063706410648065106540688
:100D14000FEF0BBB01E008BB08EF05BB002702BBCC
:100D24000ABB02E107BB07E004BB08EF01BB03E316
:100D340009B90CE10AB901E00EBD002708B901E0C8
:020D4400089510
:100D46000091DE01003064F50091DF0101FF0AC069
:100D560028D00D7F0093DF0178940091E001109177
:100D6600E1010DC00091DF0100FF1AC01AD00E7F0D
:100D76000093DF0178940091E2011091E301209144
:100D86002001239527702093200114D0E0912001A3
:100D9600FF27EE0FFF1FE050FF4F208331830FD058
:100DA60008950091DE010F770093DE01F89400911B
:100DB600DF0108952091A0013091A10108950093CB
:100DC600A0011093A101089506E010E031DB009325
:100DD600A40107E010E02CDB00939C0108E010E082
:100DE600EEDF0091A40104FF02C003E001C000276A
:100DF60008B9B3DC88D9002309F4D3D940CC83D809
:100E0600C19AC49A06EE0093A201DEDF7894579A3F
:100E160009B7006809BF439AC19AC49802C0C1982D
:100E2600C49A45DF0091A301063E79F496DC01964B
:100E3600883E03E09007A8F3C49888279927C19BAA
:100E460002C0C198EECFC19AECCF7ADF0091A4011F
:100E560003FF13C00091A201063EF1F20091E501E5
:100E66001091E601A7DF0217130781F406EE00933F
:100E7600A20102E00093A601CFCF02E010E0D8DA8B
:100E86000093A2010091A201063E31F201D4C7CF20
:100E96008A93802F40D000ED04D0082F02D089918C
:100EA600089574D058C00027F3DF35D001ED6ED019
:100EB6005CD07DD000938F0161D079D000939001F2
:100EC6005DD075D00093910159D071D000939201F5
:100ED6005AD039C00027DCDF00918F01E2DF009194
:100EE6009001DFDF00919101DCDF00919201D9DFF3
:0C0EF6002AC007E0CDDF00E8D4DF25C0F3
:100F0200002311F00A95FCCF089504D0979804E0CD
:100F1200F7CF8E9A979A04E0F3CF8A9397988E9898
:100F22008AE0869B06C0969AF4DF9698F4DF97983B
:100F320004C0EBDF8A95A9F702D089910895009148
:100F4200A50101600093A501089597989698E1DFA5
:100F5200969AE1DF97988E9808958A938E988827BB
:100F6200869B8FEFD2DF8E9A082F899108958A93FC
:100F72008E988827869B8FEFC8DF082F8991089566
:100F820096988E9AC2DF8E980895969A8E9ABDCFC1
:100F9200BCD7802F98E09A9501E0492F3DD70823CE
:100FA20011F0969A01C09698B0DF9923A1F7E2E07A
:100FB200BDC7ABD788E08A95869B05C001E0482F64
:100FC2002BD7902B05C001E0482F26D70095902300
:100FD2009CDF882381F7092FE2E0A8C796D7802FEC
:100FE200912F08D0092FD4DFB8DF082FD1DFB5DF6A
:100FF200E2E09CC792DF00EACBDFAFCF86D7A5DF66
:1010020084E690E0082F092B29F0F4DF002319F47D
:101012000197F8CF94DF99DFE2E088C774D7942F65
:101022002C813D81A22FB32FD9DF77DF01EAB0DF18
:101032009EDF8827BEDFE82FFF27EA0FFB1F008312
:1010420083959A9511F09CDFF5CF9FDF7EDFE6E076
:101052006BC757D7802F912FB42F0E811F81402E3F
:10106200512EAA27082F192FB9DFEA2FFF27E40DE7
:10107200F51D00818DDF71DFBA95A3950196BB2323
:1010820011F4BCDF05C0082F0F7179F7B7DFEACF83
:04109200E8E048C783
:1010960000919F01039500939F010091C301109158
:1010A600C40102FD0FC00091C30100FF02C0A99A4E
:1010B60001C0A9980091C30101FF02C0A89A089532
:1010C600A898089500919F0103FDEDCFA998A898CF
:0210D60008957B
:1010D800202F312F220F331F43E0B5D6200F311FA9
:1010E800022F132F08950A921A922A923A920A937B
:1010F8001A932A933A934A935A936A937A93EA9360
:10110800FA93FFB7FA939A938A9300E870D0009104
:10111800C1011091C201053620E0120710F004E663
:1011280010E02091A40124FF3BC020918801309158
:101138008901232BE9F42227E02FF12F3A9720F099
:101148000A5010402395F8CFE22FFF27EE0FFF1F1C
:10115800E855FF4FC895002D3196C8950093860134
:101168000092870100E012E0009388011093890142
:1011780000918801109189012091860130918701A1
:1011880002231323012B11F000EC31D0E8E8F1E041
:10119800008111811695079500831183449A14C024
:1011A80097DF96DF000F111F000F111F2AE43CE99B
:1011B800201B310B022F132F20EC2FBD2CB53DB572
:1011C800200F311F3BBD2ABD89919991F991FFBF2D
:1011D800F991E991799169915991499139912991B7
:1011E80019910991399029901990099018950FBD76
:0C11F8008CB59DB50A969BBD8ABD08957C
:020018006AC8B4
:1000A80000000002100244029402AA02B502DB0218
:0600B800DE03EF03FF036D
:101204000091A40100FF12C023B309B31127009376
:10121400CD012093CE01EDECF1E000919D0107D0CA
:101224000DD00091930111D0202B08D00895009582
:101234001095208131812023312308952083318327
:10124400089506D00081118108D02081318108954C
:10125400E091CF01F091D0010895E091D101F09196
:10126400D201089508EC002311F00A95FCCF0895EB
:101274004BD684EF91E0082F092B31F0AA9AF2DFC4
:10128400AA98F0DF0197F7CFE2E04FC6007F0695FA
:1012940006950695005A11270093CF011093D001AB
:1012A40008950CD012D014D00035104008F00FE48B
:1012B400000FF0CF10D00093DA0110D00091DA01C2
:1012C400E5CF3AD00091DB01E1DFC2CF0BD0C5DF1F
:1012D400008111810895042D152DABC80FEF401A1C
:1012E400500A08950091DA010F70000F005A112777
:1012F4000093D1011093D2010895E8DF0035104026
:10130400A0F30FE4F2CF0091D90104FF04C00091CF
:10131400DA0109D002C04091DA014F7001E010E017
:1013240006D093D504C0E0DF98DF40810895009390
:10133400D7011093D80108950091D90103FF04C087
:101344000091DB01F0DFE9CF4091DB01E6CF1A9396
:101354000A933AD0013021F40881198156D832C059
:10136400083038F4F894288139813CD067DF7894C8
:1013740029C0083039F4088119810093CD011093F4
:10138400CE0120C0093029F408810BBB198115BB9B
:1013940019C00A3029F408810ABB198114BB12C090
:1013A4000B3051F424D094DF0034104058F40881F9
:1013B4004CDF24D000A306C00C3021F40C2F1D2FC9
:1013C40007D046DE229608950091DA0144E028C54C
:1013D4001A930A9342E0E0E6FF2700811127000FE9
:1013E400111F0895E02F0DD0E354FE4F0895E0E659
:1013F400FF2708952091CF013091D001E22FF32FE0
:101404000895FF27EE0FFF1F0895013031F4D5D75B
:101414000091BF011091C00138C0083030F4F89435
:10142400E1DF56DF32D078940895083031F4E8DEF5
:101434000091CD011091CE0128C0093021F425B3CB
:10144400322F0BB305C00A3041F424B3322F0AB350
:101454000093D3013093D40108950B3079F4C7DF9E
:1014640037DF0034104028F0F093D301F093D40117
:10147400089511810FD000A1112707C00C3021F469
:1014840003ED11E0A5DFC9DD08950093D3011093A6
:10149400D4010895E02FF12F089596DFB6CF00917F
:1014A400DA010F70B2CF0091DB0144E0B9D4ADCFC3
:1014B40029D5802F912FA091DA01AF70AE3030F48E
:1014C400BB27A093D501B093D60114C0082F192FC0
:1014D400B0D711270093D5011093D6010196AE30F1
:1014E40049F0082F192FA5D7E5EDF1E0AEDE302B3A
:1014F400A5DE019605ED11E0FBDE082F192FE4E0CF
:1015040012C51091DC0110FF0EC01091D90116FF15
:1015140004C01091DD01102303C01091DD01102BD4
:101524001093DD0108950093DD010091DC01016059
:101534000093DC010895002321F483DE25D011F10A
:101544001FC0013021F47DDE1FD0E1F419C0023048
:1015540021F477DE19D0A4F415C0033029F471DE28
:10156400201731076CF00EC0043029F46ADE20170E
:10157400310734F407C0053019F463DE05D014F4E0
:10158400002708950FEF0895021713070895BCD498
:10159400002319F49CDE99DE63C0013041F495DE2A
:1015A40062D052DE77DF94DE020F131F59C002307F
:1015B40041F48BDE58D048DE6DDF8ADE021B130B4C
:1015C4004FC0033039F452D083DE57D0408151816B
:1015D4002CD408C0043049F449D07ADE4ED040817E
:1015E400518155D4E82FF92F3BC0053059F43ED032
:1015F4006FDE43D0408151814AD4E82FF92F4083D4
:1016040051832FC0063041F460DE2DD01DDE42DF51
:101614005FDE0223132324C0073041F456DE23D0B7
:1016240013DE38DF55DE022B132B1AC0083041F4C9
:101634004CDE19D009DE2EDF4BDE0227132710C043
:10164400093031F4D7DE44DE18D04081FED307C020
:101654000A3039F4CFDE3CDE10D04081FCD3CEDE3C
:1016640015D0E2E062C40E2F1F2F08958091CF01A0
:101674009091D001E82FF92F0895EFCD2091D70153
:101684003091D80102231323012B08950083118381
:10169400089535D400270093DC010FEF0093DD019A
:1016A4004090A0015090A101662415DE0093D90159
:1016B4000091D901007E003E39F4662009F04CC245
:1016C40001E0602EA6C148C20091D901007F003D0F
:1016D40039F4662009F040C201E0602E1DC13CC20D
:1016E40059D2003449F4662019F403E0602E63C033
:1016F40002E0601651F030C24DD251F4662021F060
:1017040002E0601609F028C202E0602E08C024C27C
:1017140003E0602E3FD2003809F44DC0FDC02BD247
:10172400A091D901A770A6300091D901D8F403FF84
:1017340002C0D8DD01C028D2B091D901B07311F430
:10174400BDDD0DC0B03111F4ACDD09C0B03209F01B
:10175400ACCFA3DE03ED11E09FDD01C0A6CF0A2FBD
:10176400EADE27C005FF05C019D21AD287DF49F087
:1017740006C0C9DDA3DDA9DDABDD80DF11F0A1E08A
:1017840001C0AA270091D90100FF06C0F9D199DD53
:101794009FDD74DF39F004C00091D90103FF02C05A
:1017A400B1E001C0BB27AB1711F4AFEF01C0AA270A
:1017B4000A2FA7DE7ACFDFD10091D901A091D901F8
:1017C40005FD42C0AF70AD30A0F40091D90104FF13
:1017D40002C088DD01C0D8D1E8D109F466CFAB30AE
:1017E40011F45FDD14C0AC3011F471DD7CC066DD32
:1017F40028C0DBD109F459CF61DDAD3051F400913B
:10180400D90104FF03C04BDECBD120C176DDAA276A
:1018140018C0AE3041F40091D90104FD46CF56DD25
:101824000095109513C1AF3061F45CDD0091D901CE
:1018340024DF04FF03C04CDD012F01C049DD112763
:1018440005C10A2FA4DE31CFA770A33008F498D1C4
:10185400ACD109F42ACFAA2321F433DD808191810C
:1018640008C0A13081F468DD1EDE8091D30190911F
:10187400D401A1D18023912346DD20DD892B25DDF0
:101884009AD1E9F017C0A23059F41BDD808191810F
:1018940092D18023912382D1892B8BD109F11BC052
:1018A400A33079F430DD0ADD0091D9010EDD03FFA8
:1018B40005C081D1CADC202B312B20C07CD1B7DC00
:1018C4001DC0A43091F46AD10091D901E3EDF1E097
:1018D40003FF05C070D1B9DC202B312B02C06BD1C2
:1018E400A6DCACDC5DD133DDE0CEA53049F40BDD04
:1018F400E5DCEBDC60D1A9DC202731279FDCD5CEE9
:10190400A63009F0D2CE4AD154D19FDC202731270A
:1019140095DC46D11CDDC9CE53D1AF70A430F8F5A7
:1019240044D109F4C2CEAA2311F4A2DCBECEA13064
:1019340041F55DDD008D118D0093A7011093A80181
:10194400ACE0BB27A03178F43FD10081EB2FE75501
:10195400FE4F008339D1BCDCEB2FE655FE4F1083DC
:10196400A395BE5FEFCFF8940091C5010093B10138
:101974000091C5011091C6011093B201789441D42D
:1019840094CEA23009F091CE0091A7011091A80144
:101994002EDD208D318DF8DD61F687CE86CEECD03C
:1019A40004D109F482CE0A2F0E70B02F882799270C
:1019B400A0FD91E0B43059F0B63079F400912001E3
:1019C400039507700093200104D140825182409016
:1019D400DA015524480E591E68CEA83059F46EDC3D
:1019E4000091210103950770009321016EDC70DCE6
:1019F400F6D02DC0A93009F058CE60DCF0D068DCF8
:101A040064DC44DE009121010A95077000932101F2
:101A14004CCED6D0AF71AA3009F447CEAB3019F40E
:101A2400400E501E42CEAC3009F43FCEAD3009F426
:101A340059C00A2F0E71083061F43CDC0091D901C1
:101A440000FF02C04FDC01C09FD041DC3EDC1EDE43
:101A54002CCE0A2F087149F52DDC0091D90101FF24
:101A640002C040DC01C090D08BD088279927A0FD0C
:101A740091E00091DB011127800F911FE2DBA2FFAF
:101A840009C0201731070CF010CE1FDC21DC0150F7
:101A9400104007C079DD0CF008CE17DC19DC0F5FAD
:101AA4001F4FF4DD482E592E00CEA83121F40091A9
:101AB400DE01006805C0A93131F40091DE010F7721
:101AC4000093DE01F2CDAE3009F4EFCDAF3029F052
:101AD400A03109F4EACDA13179F40091DE01006866
:101AE4000093DE0176D040805180009120010A9558
:101AF400077000932001D9CDA23181F438D0A0FD24
:101B040093958093E0019093E101F894002700936A
:101B1400C9010093CA0169D0026011C0A63121F441
:101B2400F89463D00D7F0BC0A43169F420D0A0FDDC
:101B340093958093E2019093E30114D001600093A4
:101B4400E4017894B2CDA73109F0AFCD0BD00E7F6C
:101B54000093E4017894A9CD4092A0015092A10190
:101B6400E7E0DEC1F8940091DF010E7F41C0B3DBF2
:101B7400802F9927B3CBB2DBAEDB0093DA01AECB77
:101B8400AADB0093DB01AACB042D152D91DC402E9A
:101B9400512E08950091D901007C0895B4DB7DCCC9
:101BA4000091D3011091D40108950091DD01002327
:101BB4000895E3EDF1E00091D7011091D801089563
:101BC4008DDBA091D9010895EA2FEE0FE05AFF278B
:101BD4000895E091200115DCE050FF4F0895E09155
:101BE40021010FDCE05FFE4F08950091DF010D7FBE
:0A1BF4000093DF010091E401089561
:101BFE000A931A932A939BD00F5F009381010CB125
:101C0E00519B08C0023009F085C001E097D00260F8
:101C1E0084C080C01091820111FF7CC0109181019F
:101C2E00123099F400937A01023008F478C00F3123
:101C3E0008F070C010917C01103024F410918201D4
:101C4E0010FF68C000937B016AC0109181011330B0
:101C5E0031F4093108F05EC00093840160C0109128
:101C6E008101143009F042C02091840110917A0153
:101C7E00210F2E5F201709F04DC000918401002323
:101C8E0021F00027009383014AC000917A010023BE
:101C9E0089F000917A01013011F400270DC00091F6
:101CAE0084010093850100917C0100684CD00027CF
:101CBE0000937E0100917E0100937D0100918201CF
:101CCE0000FF04C000917C01006403C000917C0100
:101CDE000F7B00937C01509800917C010CB9009110
:101CEE007C01009383015498569A14C0109184017C
:101CFE001C5F20918101121740F0E0918101FF27B6
:101D0E00E35EFE4F00832ED00AC0109183011017A0
:101D1E0009F4BBCF002712D00D7F00938201F991F9
:101D2E00FFBFF991E9912991199109911895EA93BB
:101D3E00FA93FFB7FA930091810108950093810100
:101D4E0000918201089500937C01009182010E7F23
:101D5E00009382010895E0918101FF27E95CFE4F17
:101D6E000081089510918301100F1093830108953F
:101D7E000A931A93DCDF0395009381010091810190
:101D8E00013031F400917D010CB900917D0114C038
:101D9E0000918101023039F4009183010CB90027C2
:101DAE000093830124C000917D01002369F026D0A9
:101DBE0028F4D1DF0CB9CFDFD5DF19C01FD021F445
:101DCE00009183010CB913C0549A56980CB11CB1F2
:101DDE0000917C0106FF08C000917A01002321F4D6
:101DEE0000917C010F77AFDF002700938101F991FD
:101DFE00FFBFF991E991199109911895009181010F
:0A1E0E00035010917D0101170895A3
:02001200F5CD2A
:02001600B3CE67
:020000000EC030
:10001A0000EC05BFCBE2D2E00FE503500DBF02E0D2
:10002A0000400EBF72D6002309F41FD0E0E6F0E0CC
:10003A0000E010E050DFE8E7F0E000E610E040E022
:10004A0050E03BDFE0E0F1E00BEE10E044DFE8E7F0
:10005A00F0E000E011E040E050E02FDFE8E7F0E0F8
:0E006A000BEE11E040E050E028DFC7D6D0CE0C
:021E1800FFCFFA
:0A1E1A004A9512F0000FE1F7089559
:0A1E24004A9512F00695E1F70895C3
:101E2E00002411240030010741F01695079510F497
:101E3E00040E151E440F551FF5CF002D112D0895BC
:0C1E4E004A951AF0000F111FFBCF0895F9
:0C1E5A004A951AF015950795FBCF0895E6
:101E660000241124E0E1EA9552F0001F111F001C26
:101E7600111C04161506B8F3041A150AF4CF001F30
:0C1E8600111F402D512D0095109508955E
:101E9200FF27552322F4F1605195419550401123BB
:101EA20022F4F095119501951040DCDFF69518F4B7
:101EB200119501951040F69518F4519541955040B1
:021EC200089581
:101EC400BF93AF93A02FB12F03C0C89531960D9245
:0C1ED40041505040D0F7AF91BF910895ED
:0E1EE000002401C0019201501040E0F7089567
:021EEE000000F2
:101EF000FA92EA92DA92CA92BA92AA929A928A9242
:101F00007A926A925A924A92BA93AA939A938A932D
:021F1000089532
:101F1200FF84EE84DD84CC84BB84AA849984888483
:101F22007F806E805D804C80BB81AA81998188818F
:0E1F3200F0E00FB6F894CE0FDF1F0FBE08953B
:00000001FF
